:020000040000FA
:10000000FF23831690000C280515B10B0828302813
:10001000311C05110C10090083128501073099006D
:1000200083169F0138308500831207308500B01099
:1000300005116920051569200511692005156F2036
:10004000851E26286F20051E2F281F280510B01892
:100050004C206F20851E2928073085001F284C2042
:1000600005100000851005114D206920051EB014F3
:100070007520851D44280000851E40280000382872
:10008000073085004C201F2807308500B018492014
:100090001F28B01450200800B01010108B13080057
:1000A0000630B1008F018E01313090000C108316A4
:1000B0000C1483120B178B1708001930A40063204F
:1000C000A40B5F2808002830A3006F20A30B65282D
:1000D00008000C30A5006F20A50B6B280800F93034
:1000E000A1007520A10B712808001730A2000000A4
:0600F000A20B77280800B6
:02400E00C43FAD
:00000001FF
